BL51 BANKED LINKER/LOCATER V6.22.2.0                                                    03/16/2023  09:25:09  PAGE 1


BL51 BANKED LINKER/LOCATER V6.22.2.0, INVOKED BY:
C:\KEIL_V5\C51\BIN\BL51.EXE .\Release\system_FE81001.obj, .\Release\STARTUP.obj, .\Release\main.obj TO .\Release\Sample_
>> DrvRTC REGFILE (.\Release\Sample_DrvRTC.ORC) PRINT (.\Sample_DrvRTC.m51) RAMSIZE (256) CODE (0X0000-0X1FFF) XDATA (0X
>> 8000-0X87FF)


MEMORY MODEL: SMALL


INPUT MODULES INCLUDED:
  .\Release\system_FE81001.obj (SYSTEM_FE81001)
  .\Release\STARTUP.obj (?C_STARTUP)
  .\Release\main.obj (MAIN)
  C:\KEIL_V5\C51\LIB\C51S.LIB (?C_INIT)
  C:\KEIL_V5\C51\LIB\C51S.LIB (?C_IBP)


LINK MAP OF MODULE:  .\Release\Sample_DrvRTC (SYSTEM_FE81001)


            TYPE    BASE      LENGTH    RELOCATION   SEGMENT NAME
            -----------------------------------------------------

            * * * * * * *   D A T A   M E M O R Y   * * * * * * *
            REG     0000H     0008H     ABSOLUTE     "REG BANK 0"
            DATA    0008H     0004H     UNIT         ?DT?MAIN
            DATA    000CH     0002H     UNIT         ?DT?DELAY?MAIN
            DATA    000EH     0002H     UNIT         ?DT?RTCISR?MAIN
            DATA    0010H     0001H     UNIT         ?C?LIB_DATA
            IDATA   0011H     0001H     UNIT         ?STACK

            * * * * * * *   C O D E   M E M O R Y   * * * * * * *
            CODE    0000H     0003H     ABSOLUTE     
            CODE    0003H     002EH     UNIT         ?PR?CLKCONFIG?MAIN
            CODE    0031H     0001H     UNIT         ?PR?SYSTEMINIT?SYSTEM_FE81001
                    0032H     0001H                  *** GAP ***
            CODE    0033H     0003H     ABSOLUTE     
            CODE    0036H     009DH     UNIT         ?C_C51STARTUP
            CODE    00D3H     008BH     UNIT         ?PR?RTCISR?MAIN
            CODE    015EH     004EH     UNIT         ?PR?IOCONFIG?MAIN
            CODE    01ACH     003EH     UNIT         ?PR?RTCCONFIG?MAIN
            CODE    01EAH     001EH     UNIT         ?PR?MAIN?MAIN
            CODE    0208H     001CH     UNIT         ?PR?DELAY?MAIN
            CODE    0224H     0009H     UNIT         ?C_INITSEG



OVERLAY MAP OF MODULE:   .\Release\Sample_DrvRTC (SYSTEM_FE81001)


SEGMENT
  +--> CALLED SEGMENT
---------------------
?C_C51STARTUP
  +--> ?PR?MAIN?MAIN
  +--> ?C_INITSEG

?PR?MAIN?MAIN
BL51 BANKED LINKER/LOCATER V6.22.2.0                                                  03/16/2023  09:25:09  PAGE 2


  +--> ?PR?CLKCONFIG?MAIN
  +--> ?PR?IOCONFIG?MAIN
  +--> ?PR?RTCCONFIG?MAIN

?PR?CLKCONFIG?MAIN
  +--> ?PR?DELAY?MAIN



SYMBOL TABLE OF MODULE:  .\Release\Sample_DrvRTC (SYSTEM_FE81001)

  VALUE           TYPE          NAME
  ----------------------------------

  -------         MODULE        SYSTEM_FE81001
  C:0000H         SYMBOL        _ICE_DUMMY_
  C:0031H         PUBLIC        SystemInit
  -------         PROC          SYSTEMINIT
  C:0031H         LINE#         38
  C:0031H         LINE#         39
  C:0031H         LINE#         41
  -------         ENDPROC       SYSTEMINIT
  -------         ENDMOD        SYSTEM_FE81001

  -------         MODULE        ?C_STARTUP
  C:0036H         SEGMENT       ?C_C51STARTUP
  I:0011H         SEGMENT       ?STACK
  C:0000H         PUBLIC        ?C_STARTUP
  D:00E0H         SYMBOL        ACC
  D:00F0H         SYMBOL        B
  D:0083H         SYMBOL        DPH
  D:0082H         SYMBOL        DPL
  N:0001H         SYMBOL        IBPSTACK
  N:0100H         SYMBOL        IBPSTACKTOP
  N:0080H         SYMBOL        IDATALEN
  C:0039H         SYMBOL        IDATALOOP
  N:0000H         SYMBOL        PBPSTACK
  N:0100H         SYMBOL        PBPSTACKTOP
  N:0000H         SYMBOL        PDATALEN
  N:0000H         SYMBOL        PDATASTART
  N:0000H         SYMBOL        PPAGE
  N:0000H         SYMBOL        PPAGEENABLE
  D:00A0H         SYMBOL        PPAGE_SFR
  D:0081H         SYMBOL        SP
  C:0036H         SYMBOL        STARTUP1
  N:0000H         SYMBOL        XBPSTACK
  N:0000H         SYMBOL        XBPSTACKTOP
  N:0800H         SYMBOL        XDATALEN
  C:0044H         SYMBOL        XDATALOOP
  N:8000H         SYMBOL        XDATASTART
  C:0000H         LINE#         126
  C:0036H         LINE#         133
  C:0038H         LINE#         134
  C:0039H         LINE#         135
  C:003AH         LINE#         136
  C:003CH         LINE#         140
  C:003FH         LINE#         141
BL51 BANKED LINKER/LOCATER V6.22.2.0                                                  03/16/2023  09:25:09  PAGE 3


  C:0041H         LINE#         145
  C:0043H         LINE#         147
  C:0044H         LINE#         148
  C:0045H         LINE#         149
  C:0046H         LINE#         150
  C:0048H         LINE#         151
  C:004AH         LINE#         170
  C:004DH         LINE#         185
  C:0050H         LINE#         196
  -------         ENDMOD        ?C_STARTUP

  -------         MODULE        MAIN
  C:0000H         SYMBOL        _ICE_DUMMY_
  D:0090H         PUBLIC        P1
  D:00B0H         PUBLIC        P3
  D:00A8H         PUBLIC        IE
  C:0208H         PUBLIC        delay
  D:00B8H         PUBLIC        IP
  C:01EAH         PUBLIC        main
  D:0008H         SYMBOL        clb_data
  D:0098H         PUBLIC        SCON
  C:0003H         PUBLIC        CLKConfig
  D:0088H         PUBLIC        TCON
  C:01ACH         PUBLIC        RTCConfig
  D:000BH         SYMBOL        cnt
  C:00D3H         PUBLIC        RTCISR
  D:00C8H         PUBLIC        T2CON
  C:015EH         PUBLIC        IOConfig
  D:00D0H         PUBLIC        PSW
  -------         PROC          DELAY
  -------         DO            
  D:000CH         SYMBOL        i
  -------         ENDDO         
  C:0208H         LINE#         35
  C:0208H         LINE#         36
  C:0208H         LINE#         39
  C:0223H         LINE#         40
  -------         ENDPROC       DELAY
  -------         PROC          RTCISR
  -------         DO            
  D:000EH         SYMBOL        int_stat
  -------         ENDDO         
  C:00D3H         LINE#         52
  C:00E2H         LINE#         54
  C:00EDH         LINE#         57
  C:00F2H         LINE#         58
  C:00F8H         LINE#         60
  C:0105H         LINE#         62
  C:0105H         LINE#         64
  C:010AH         LINE#         65
  C:0110H         LINE#         67
  C:0110H         LINE#         70
  C:0115H         LINE#         71
  C:011BH         LINE#         73
  C:011BH         LINE#         76
  C:0120H         LINE#         77
  C:0126H         LINE#         79
BL51 BANKED LINKER/LOCATER V6.22.2.0                                                  03/16/2023  09:25:09  PAGE 4


  C:0133H         LINE#         80
  C:0133H         LINE#         83
  C:0138H         LINE#         84
  C:013EH         LINE#         86
  C:014BH         LINE#         87
  C:014BH         LINE#         91
  C:0151H         LINE#         92
  -------         ENDPROC       RTCISR
  -------         PROC          RTCCONFIG
  C:01ACH         LINE#         104
  C:01ACH         LINE#         105
  C:01ACH         LINE#         107
  C:01B2H         LINE#         108
  C:01B8H         LINE#         109
  C:01BEH         LINE#         110
  C:01C3H         LINE#         113
  C:01C9H         LINE#         114
  C:01CFH         LINE#         115
  C:01D5H         LINE#         118
  C:01DBH         LINE#         121
  C:01E1H         LINE#         124
  C:01E9H         LINE#         125
  -------         ENDPROC       RTCCONFIG
  -------         PROC          IOCONFIG
  C:015EH         LINE#         137
  C:015EH         LINE#         138
  C:015EH         LINE#         140
  C:0169H         LINE#         143
  C:018AH         LINE#         146
  C:01ABH         LINE#         147
  -------         ENDPROC       IOCONFIG
  -------         PROC          CLKCONFIG
  C:0003H         LINE#         159
  C:0003H         LINE#         160
  C:0003H         LINE#         162
  C:0011H         LINE#         165
  C:001CH         LINE#         168
  C:002DH         LINE#         171
  C:0030H         LINE#         172
  -------         ENDPROC       CLKCONFIG
  -------         PROC          MAIN
  C:01EAH         LINE#         184
  C:01EAH         LINE#         185
  C:01EAH         LINE#         186
  C:01EDH         LINE#         187
  C:01F0H         LINE#         189
  C:01F3H         LINE#         191
  C:01F9H         LINE#         192
  C:01FFH         LINE#         193
  C:0205H         LINE#         197
  C:0205H         LINE#         198
  C:0205H         LINE#         207
  -------         ENDPROC       MAIN
  -------         ENDMOD        MAIN

  -------         MODULE        ?C_IBP
  D:0010H         PUBLIC        ?C_IBP
BL51 BANKED LINKER/LOCATER V6.22.2.0                                                  03/16/2023  09:25:09  PAGE 5


  -------         ENDMOD        ?C_IBP



FUNCTION REGISTER MASKS


FUNCTION . . . . . REG MASK
---------------------------

CLKCONFIG. . . . . @0xf303
DELAY. . . . . . . @0xf000
IOCONFIG . . . . . @0xe301
MAIN . . . . . . . @0xf303
RTCCONFIG. . . . . @0xe301
RTCISR . . . . . . @0xe303
SYSTEMINIT . . . . @0x8000

*** WARNING L16: UNCALLED SEGMENT, IGNORED FOR OVERLAY PROCESS
    SEGMENT: ?PR?SYSTEMINIT?SYSTEM_FE81001

Program Size: data=18.0 xdata=0 code=556
LINK/LOCATE RUN COMPLETE.  1 WARNING(S),  0 ERROR(S)
